:1000000027C03FC03EC03DC03CC03BC03AC039C025
:1000100038C037C036C035C034C033C032C031C03C
:1000200030C02FC02EC01E910862DFFF1E920662F4
:10003000DFFF1E930B62DFFF1E90076AFF001E901A
:10004000045200001E90051C00000000000000008B
:1000500011241FBECFEDCDBF80E288BB8FE787BBE9
:100060008CE182BB80E481BB10E0A0E6B0E0ECE371
:10007000F3E002C005900D92A236B107D9F750D037
:100080005BC1BECF482FC098C198C39A0000C398E7
:1000900020E030E086B3220F90E096958795969504
:1000A00087958170282B47FF02C0C09A01C0C09875
:1000B00067FF02C0C19A01C0C198C39A0000C398EB
:1000C0003F5F383019F0440F660FE4CFC098C198F5
:1000D000C39A0000C398C39A0000C398822F089562
:1000E00080E090E036E0B2990AC0232F2A95F1F71C
:1000F000019623E0883E9207B1F7109260000895C0
:100100001F93182F88E06CE4BDDF812F6CE0BADF0D
:1001100080E068E6B7DF80E06CE6B4DF1F91089509
:10012000EF92FF920F931F93CF93DF9380E18A9515
:10013000F1F780E388BB8DE08A95F1F780E588BB15
:1001400085E08A95F1F7BA9884E68A95F1F700E0A0
:1001500023C080E0D5DF8117F1F481E0D1DF282FC3
:10016000802F90E066E070E0D5D0FC01E95DFF4FA4
:10017000E4912E1781F482E0C3DF282F802F90E0D6
:1001800063E070E0C7D0FC01EE0FFF1FE85DFF4F9A
:10019000E4912E1761F00F5F802F90E066E070E031
:1001A000B9D0FC01EA5DFF4F1491112391F6802F25
:1001B00090E066E070E0AED0EC01CA5DDF4FFE017A
:1001C0008491882309F46DC0802F90E066E070E090
:1001D000A1D0FC01E75DFF4FF490802F90E066E036
:1001E00070E098D0FC01E65DFF4F1491802F90E005
:1001F00066E070E08FD0FC01E55DFF4FE49080B3D6
:1002000084FF02C0033088F080E86CE43BDF80E0CC
:1002100064E638DF80E06CE635DF62DF80E06CE4C6
:1002200031DF5EDFFF20B9F004C082FF70C01DED3A
:100230006FC00F2D80E46CE425DF802F6CE222DF9D
:1002400080E064E61FDF80E06CE61CDF49DF80E0D1
:100250006CE418DF45DF112389F080E46CE412DFE1
:10026000812F6CE20FDF80E064E70CDF80E06CE759
:1002700009DF36DF80E06CE405DF32DFEE2089F055
:1002800080E46CE4FFDE8E2D6CE2FCDE80E066E64E
:10029000F9DE80E06EE6F6DE23DF80E06CE4F2DE7D
:1002A0001FDF86E08A95F1F780E388BB81E08A95BD
:1002B000F1F780E288BB969A80916000882351F420
:1002C00080E197E229E130E0F9013197F1F70197F8
:1002D000D9F712C0FE018491882351F488EB9BE08A
:1002E00029E130E0F9013197F1F70197D9F704C01E
:1002F00088EA91E60197F1F7969885B7806585BF02
:1003000085B7806285BF889585B78F7DF8CF1DE55D
:1003100001EE90CF5527002480FF02C0060E571F24
:10032000660F771F6115710521F0969587950097E7
:0C03300099F7952F802D0895F894FFCFC9
:02033C000100BE
:00000001FF
